:020000040000FA
:04000000F1EF00F02C
:02000800FDD029
:0800180053D10A6A0C6A0B6E59
:10002000010E056E0C500A5C02E10B50095C040ED7
:10003000D8B0010ED8B4020E0514D8A4010E1200D7
:100040000F0EEA6E02C0E9FF0350E988E92AEC12BC
:1000500002C0E9FFF40E0F6E010E106EA4D80A2A3A
:10006000092A0E2A0B6A0C6AEF5003140F6E000067
:10007000EF50031403180F12D8B40B2AD8B40C2A6B
:1000800003180F6E0D06D8B40E06D8B40906D8B4FE
:100090000A2EEDD70B501200126E960E096E980EB6
:1000A0000A6E6AD8D8B4CA90D8A4CA80FC0FD8A067
:1000B000CA92D8B0CA82800E096E960E0A6E980E49
:1000C0000D6E0E6ACAB025D8CAB223D857D8090413
:1000D000CB6E09C00BF00AC00CF002500F6E106E10
:1000E000023C106A60D80E50122E0AD0BE6E0C0E62
:1000F000BD6E0DBEBD8A0DBCBD889394CA8412002E
:10010000BB6E0C0EBA6E0DBEBA8A0DBCBA88949244
:10011000F5D700D8D8900D320A3209321200E836ED
:10012000E8363C0B0109C212C009C216C050F80BD8
:100130000609C06E190E15D8C282C2B2FED7C4CF4E
:1001400015F0C350146E12000C6A0B6EFF0E0B26D6
:100150000C2200D0D8A01200030E0A6EE70E02D8BF
:10016000F5D70A6AFE0F096EE86A0A5AD8A012008B
:100170000000090600D0F8D70E6A0D6A100EF36E63
:100180000A340D360E360B500D5C0C500E5805E33C
:100190000B500D5E0C500E5AD88009360A36F32EDD
:1001A000EFD7095012000B500F02F4CF0EF0F3CF2F
:1001B0000DF00C501002F4CF0AF0F3CF09F00B5001
:1001C0001002F3500E26F4500922E86A0A220C505D
:1001D0000F02F3500E26F4500922E86A0A220D504D
:1001E0001200F86A006A4F0EAF6E240EAC6E900ECD
:1001F000AB6E0001C69A810E926EC10E936EC00E58
:10020000946ED1D09EAA1BD0060EAB1412E1E1CFA2
:1002100050F0E2CF51F0522A1EEE80F05250E1260B
:10022000000EE222AECFE7FF50C0E1FF51C0E2FF77
:100230001100AE50AE50AB98AB88110011D0F2A4B3
:1002400009D0F294194A1A2A817A186AD6CF17F07F
:10025000110006D0F2A204D0F2924C4A4D2A1100AD
:1002600011005250535C14E0532AE9CF09F0EACF51
:100270000AF00EEE80F05350E926000EEA22EF500D
:10028000096E09C0E9FF0AC0EAFFD880120004D055
:10029000E868096ED8A012001200526A536A9D8A5B
:1002A0009F8AF28EF28CF28A12009D9A0EEE80F0F6
:1002B000000EEE6AE82EFDD7526A536A9D8A12003C
:1002C000F29ED8CF54FEE8CF55FEE0CF56FEE9CFE0
:1002D00057FEEACF58FEE1CF59FEE2CF5AFED9CF02
:1002E0005BFEDACF5CFEF6CF5DFEF7CF5EFEF5CFAC
:1002F0005FFEF3CF60FEF4CF61FEA6CF62FE09C0C1
:1003000063FE0AC064FE0FC065FE11C066FE14C025
:1003100067FE15C068FEF28E0001A1922B0EB26E30
:10032000CF0EB36E4B2A640E4B5C07E14B6A4CC098
:1003300047F04DC048F04C6A4D6A000EF0DE416E49
:1003400015C042F0F29E54CED8FF55CEE8FF56CEEF
:10035000E0FF57CEE9FF58CEEAFF59CEE1FF5ACE73
:10036000E2FF5BCED9FF5CCEDAFF5DCEF6FF5ECE5C
:10037000F7FF5FCEF5FF60CEF3FF61CEF4FF62CEF4
:10038000A6FF63CE09F064CE0AF065CE0FF066CE0C
:1003900011F067CE14F068CE15F0F28E10009EA812
:1003A000FED7AD6E1200939A8A9A949A8B9A94987B
:1003B0008B9892988998929A898A93968A86939430
:1003C0008A9493928A829294898492968986026A08
:1003D000280E0B6E260E0C6E010E5EDE026A280ED3
:1003E0000B6E260E0C6E020E57DE270E356E4E0E6D
:1003F0004E6E1E0E456E030E466E366A010E376E49
:10040000396A400E3A6E030E3B6E400E3C6EFA0E99
:100410009BDE8988898A386838C002F0280E0B6E06
:10042000260E0C6E020E38DE030E0C6EE80E8DDE0C
:10043000386A38C002F0280E0B6E260E0C6E020EC3
:100440002BDE939A8A8A320E7FDE939A8A9A336AD7
:10045000346A23DF2ADFCD6AF294F28A870ED56EE2
:10046000F292F2888E0EC06E0E0EC16E010EC26E3A
:10047000B16AA192A082B26AB36AD08EA292B10E82
:10048000B16EEFDE1B6EBB0E1B5C05E3FE0E1B5C4C
:1004900001E21E6AE8D01BAE21D01E6A8A0E1B5CE8
:1004A00005E11BC01EF01F68206817D09A0E1B5C68
:1004B00005E11BC01EF0216822680FD0AA0E1B5C4C
:1004C00005E11BC01EF02368246807D0BA0E1B5C30
:1004D00004E11BC01EF025682668C5D01E5202E14B
:1004E000C2D0C1D08A0E1E5C31E11F2803E11BC0BF
:1004F0001FF02AD01BC020F07E0E1F5C04E189840F
:1005000033944F9420D07F0E1F5C04E1898633968C
:100510004F9619D0270E1F5C0CE0330E1F5C09E0CC
:100520003F0E1F5C06E04B0E1F5C03E0570E1F5C86
:1005300003E14F80899A07D0280E1F5C04E3570E11
:100540001F5CD8A0899A1F688ED08DD09A0E1E5C31
:10055000D8A470D0212803E11BC021F069D01BC0B2
:1005600022F022522AE17E0E215C04E18984339438
:100570004F9420D07F0E215C04E1898633964F96FC
:1005800019D0270E215C0CE0330E215C09E03F0EF0
:10059000215C06E04B0E215C03E0570E215C03E179
:1005A0004F80899A07D0280E215C04E3570E215C06
:1005B000D8A0899A216857D03AD0270E215C0CE048
:1005C000330E215C09E03F0E215C06E04B0E215CFE
:1005D00003E0570E215C03E14F80898A28D0280E62
:1005E000215C06E3570E215C03E24F90898A1FD0FD
:1005F0007E0E215C0DE189944F847F0E225C02E126
:10060000339405D021C023F022C024F05DD90FD04F
:100610007F0E215C0CE189964F867F0E225C02E101
:10062000339605D021C023F022C024F04DD9216893
:100630001AD019D0AA0E1E5C0AE1232803E11BC0C0
:1006400023F003D01BC024F03FD90DD00CD0BA0E3C
:100650001E5C09E1252803E11BC025F003D01BC067
:1006600026F0A3D900D03352D8B47AD033A41AD00C
:1006700062C02DF063C02EF06CC02BF06DC02CF06A
:10068000D6CF17F0D7CF18F02B50175C2C50185836
:100690002D5019582E501A581A502E18D8B0800ABA
:1006A000D8B8CCD833A61AD064C02DF065C02EF0CF
:1006B0006EC02BF06FC02CF0D6CF17F0D7CF18F04C
:1006C0002B50175C2C5018582D5019582E501A5872
:1006D0001A502E18D8B0800AD8B8D3D833A840D032
:1006E00066C02DF067C02EF070C02BF071C02CF0EA
:1006F000D6CF17F0D7CF18F02B50175C2C501858C6
:100700002D5019582E501A581A502E18D8B0800A49
:1007100027E78B9A8B983398485207E147504E5CF5
:1007200004E18A848A968A9211D0485207E14E5099
:10073000475C04E28A948A828A9608D0485203E190
:1007400047504E5C03E28A948A868A92400E3C6E41
:100750003DAA06D0BA0E23DE330E21DE400E1FDE88
:1007600090D64FA028D0365226E0485214E1475088
:100770004E5C11E1366A8A848A968A928B9A8B98AB
:100780003752D8B4899A3DAC06D0BA0E08DE160EA0
:1007900006DE7F0E04DE485203E147504E5C06E25F
:1007A0008A868A948A928B8A8B9805D08A968A94B4
:1007B0008A828B9A8B883DA01FD04A50485C03E107
:1007C0004950475C19E07F0E47141C6E47C01DF06E
:1007D00048C0F3FF070EF3321D32E82EFCD7AA0EF5
:1007E000CFEC01F01D50CFEC01F01C50CFEC01F02C
:1007F00047C049F048C04AF03DA21FD04450425C77
:1008000003E14350415C19E07F0E41141C6E41C06E
:100810001DF042C0F3FF070EF3321D32E82EFCD765
:10082000EA0ECFEC01F01D50CFEC01F01C50CFECE4
:1008300001F041C043F042C044F023D64FB403D08E
:10084000339489841DD0D6CF17F0D7CF18F058C075
:1008500006F059C007F0065017242B6E07501820D9
:100860002C6E000E19202D6E000E1A202E6E2DC03B
:1008700062F02EC063F02BC06CF02CC06DF0807461
:1008800012004FB603D0339689861DD0D6CF17F00D
:10089000D7CF18F05AC006F05BC007F006501724F7
:1008A0002B6E075018202C6E000E19202D6E000E96
:1008B0001A202E6E2DC064F02EC065F02BC06EF095
:1008C0002CC06FF0807612007E0E235C32E14FA4C4
:1008D0002DD03384D6CF17F0D7CF18F0241C086E54
:1008E0007F0E0814146E156A14C007F0066AD890BB
:1008F000073606C058F007C059F058C006F059C076
:1009000007F0065017242B6E075018202C6E000E8F
:1009100019202D6E000E1A202E6E2DC062F02EC0F2
:1009200063F02BC06CF02CC06DF002D0339489843E
:1009300034D07F0E235C31E14FA62DD03386D6CF45
:1009400017F0D7CF18F0241C086E7F0E0814146E11
:10095000156A14C007F0066AD890073606C05AF028
:1009600007C05BF05AC006F05BC007F006501724C2
:100970002B6E075018202C6E000E19202D6E000EC5
:100980001A202E6E2DC064F02EC065F02BC06EF0C4
:100990002CC06FF002D03396898623681200276836
:1009A00012002968120028681200070E255C10E169
:1009B000D8902634386E2652D8A4382A38C002F08F
:1009C000280E0B6E260E0C6E020E4CEC00F0FAD0C8
:1009D000140E255CD8A44ED026C009F0230E0DECD1
:1009E00000F0166E2E0E265C010ED8B0E86A1616C0
:1009F00003E026C035F002D0270E356E240E355C9C
:100A000003E1410E4E6E35D0250E355C03E1450EF7
:100A10004E6E2FD0260E355C03E1490E4E6E29D066
:100A2000270E355C03E14E0E4E6E23D0280E355C4A
:100A300003E1520E4E6E1DD0290E355C03E1570EB8
:100A40004E6E17D02A0E355C03E15D0E4E6E11D04E
:100A50002B0E355C03E1620E4E6E0BD02C0E355C16
:100A600003E1680E4E6E05D02D0E355C02E16E0E70
:100A70004E6EA8D0160E255C0DE126C036F0898892
:100A8000898A0268280E0B6E260E0C6E020E4CEC44
:100A900000F098D0170E255C08E126C037F03752D9
:100AA00002E0898A01D0899A8DD0280E255C03E165
:100AB00026C039F087D0290E255C03E126C03AF024
:100AC00081D02A0E255C03E126C03BF07BD0330E9B
:100AD000255CD8A466D026C03CF0400E3C5C04E106
:100AE0008B9A8B9833985CD0400E3C5C2CE226505D
:100AF0004008266E8B9A3388D6CF17F0D7CF18F0E0
:100B0000D8903C30076E066A063206C05CF007C01B
:100B10005DF05CC006F05DC007F0065017242B6E38
:100B2000075018202C6E000E19202D6E000E1A2072
:100B30002E6E2DC066F02EC067F02BC070F02CC05A
:100B400071F08B882DD0410E3C5C2AE3400E265E6E
:100B50008B983388D6CF17F0D7CF18F0D8903C3089
:100B6000076E066A063206C05CF007C05DF05CC026
:100B700006F05DC007F0065017242B6E07501820B2
:100B80002C6E000E19202D6E000E1A202E6E2DC018
:100B900066F02EC067F02BC070F02CC071F08B8A0D
:100BA00011D0420E255C04E12652D8B41FD80AD0D9
:100BB000500E255C03E126C03DF004D07B0E255C81
:100BC000D8B402D825681200939A8A9A899A376A0B
:100BD00089848986336A346A026A280E0B6E260E6F
:100BE0000C6E020E4CEC00F0386A1200949A8B9A4C
:100BF00094988B9893968A9693928A9293948A94D7
:100C0000899A376A939A8A9A336A346A026A280EF2
:100C10000B6E260E0C6E020E4CEC00F0386A196A50
:100C20001A6A898489861200810E026E010E036E93
:100C3000E80E0B6E030E0C6E20EC00F0476E0CC03D
:100C400048F04852D8A44CD047504E5CD8A448D065
:100C50008A848A968A928B9A8B987F0E47141C6E90
:100C600047C01DF048C0F3FF070EF3321D32E82ED7
:100C7000FCD7AA0ECFEC01F01D50CFEC01F01C50B8
:100C8000CFEC01F047C049F048C04AF0416A426ADF
:100C90001C6A100E1C5C0FE2000E8FEC00F0066E5A
:100CA00015C007F006504126075042220A0EA4EC58
:100CB00000F01C2AEEE14230466E4130456E46326D
:100CC000453246324532463245320F0E4616BA0E8E
:100CD000CFEC01F0160ECFEC01F07F0ECFEF01F05C
:100CE000485203E147504E5C12E28B9A8B888A8609
:100CF0008A928A944E50475C146E000E4858156EC6
:100D000014C00CF00B6AA6EC00F08B9811D08B98F5
:100D10008B8A8A968A828A9447504E5C146E000EA3
:100D20004854156E14C00CF00B6AA6EC00F08B9AB8
:060D30007BD71200FFD783
:020000040030CA
:0300010006170ED1
:020005008580F4
:060008000FC00FE00F40E5
:00000001FF
